C51 COMPILER V9.51   S_SCLK_PIN                                                            10/14/2013 23:29:43 PAGE 1   


C51 COMPILER V9.51, COMPILATION OF MODULE S_SCLK_PIN
OBJECT MODULE PLACED IN .\DP8051_Keil_951\Debug\s_sclk_pin.obj
COMPILER INVOKED BY: C:\Program Files (x86)\Cypress\PSoC Creator\3.0\PSoC Creator\import\keil\pk51\9.51\C51\BIN\c51.exe 
                    -.\Generated_Source\PSoC3\s_sclk_pin.c NOIV LARGE MODDP2 OMF2 VB(1) PR(.\DP8051_Keil_951\Debug\s_sclk_pin.lst) CD DB NOIP
                    - OT(5,SIZE) INCDIR(.,.\Generated_Source\PSoC3) OJ(.\DP8051_Keil_951\Debug\s_sclk_pin.obj)

line level    source

   1          /*******************************************************************************
   2          * File Name: s_sclk_pin.c  
   3          * Version 1.90
   4          *
   5          * Description:
   6          *  This file contains API to enable firmware control of a Pins component.
   7          *
   8          * Note:
   9          *
  10          ********************************************************************************
  11          * Copyright 2008-2012, Cypress Semiconductor Corporation.  All rights reserved.
  12          * You may use this file only in accordance with the license, terms, conditions, 
  13          * disclaimers, and limitations in the end user license agreement accompanying 
  14          * the software package with which this file was provided.
  15          *******************************************************************************/
  16          
  17          #include "cytypes.h"
  18          #include "s_sclk_pin.h"
  19          
  20          
  21          /*******************************************************************************
  22          * Function Name: s_sclk_pin_Write
  23          ********************************************************************************
  24          *
  25          * Summary:
  26          *  Assign a new value to the digital port's data output register.  
  27          *
  28          * Parameters:  
  29          *  prtValue:  The value to be assigned to the Digital Port. 
  30          *
  31          * Return: 
  32          *  None 
  33          *  
  34          *******************************************************************************/
  35          void s_sclk_pin_Write(uint8 value) 
  36          {
  37   1          uint8 staticBits = (s_sclk_pin_DR & (uint8)(~s_sclk_pin_MASK));
  38   1          s_sclk_pin_DR = staticBits | ((uint8)(value << s_sclk_pin_SHIFT) & s_sclk_pin_MASK);
  39   1      }
  40          
  41          
  42          /*******************************************************************************
  43          * Function Name: s_sclk_pin_SetDriveMode
  44          ********************************************************************************
  45          *
  46          * Summary:
  47          *  Change the drive mode on the pins of the port.
  48          * 
  49          * Parameters:  
  50          *  mode:  Change the pins to this drive mode.
  51          *
  52          * Return: 
  53          *  None
C51 COMPILER V9.51   S_SCLK_PIN                                                            10/14/2013 23:29:43 PAGE 2   

  54          *
  55          *******************************************************************************/
  56          void s_sclk_pin_SetDriveMode(uint8 mode) 
  57          {
  58   1              CyPins_SetPinDriveMode(s_sclk_pin_0, mode);
  59   1      }
  60          
  61          
  62          /*******************************************************************************
  63          * Function Name: s_sclk_pin_Read
  64          ********************************************************************************
  65          *
  66          * Summary:
  67          *  Read the current value on the pins of the Digital Port in right justified 
  68          *  form.
  69          *
  70          * Parameters:  
  71          *  None 
  72          *
  73          * Return: 
  74          *  Returns the current value of the Digital Port as a right justified number
  75          *  
  76          * Note:
  77          *  Macro s_sclk_pin_ReadPS calls this function. 
  78          *  
  79          *******************************************************************************/
  80          uint8 s_sclk_pin_Read(void) 
  81          {
  82   1          return (s_sclk_pin_PS & s_sclk_pin_MASK) >> s_sclk_pin_SHIFT;
  83   1      }
  84          
  85          
  86          /*******************************************************************************
  87          * Function Name: s_sclk_pin_ReadDataReg
  88          ********************************************************************************
  89          *
  90          * Summary:
  91          *  Read the current value assigned to a Digital Port's data output register
  92          *
  93          * Parameters:  
  94          *  None 
  95          *
  96          * Return: 
  97          *  Returns the current value assigned to the Digital Port's data output register
  98          *  
  99          *******************************************************************************/
 100          uint8 s_sclk_pin_ReadDataReg(void) 
 101          {
 102   1          return (s_sclk_pin_DR & s_sclk_pin_MASK) >> s_sclk_pin_SHIFT;
 103   1      }
 104          
 105          
 106          /* If Interrupts Are Enabled for this Pins component */ 
 107          #if defined(s_sclk_pin_INTSTAT) 
              
                  /*******************************************************************************
                  * Function Name: s_sclk_pin_ClearInterrupt
                  ********************************************************************************
                  *
                  * Summary:
                  *  Clears any active interrupts attached to port and returns the value of the 
                  *  interrupt status register.
C51 COMPILER V9.51   S_SCLK_PIN                                                            10/14/2013 23:29:43 PAGE 3   

                  *
                  * Parameters:  
                  *  None 
                  *
                  * Return: 
                  *  Returns the value of the interrupt status register
                  *  
                  *******************************************************************************/
                  uint8 s_sclk_pin_ClearInterrupt(void) 
                  {
                      return (s_sclk_pin_INTSTAT & s_sclk_pin_MASK) >> s_sclk_pin_SHIFT;
                  }
              
              #endif /* If Interrupts Are Enabled for this Pins component */ 
 130          
 131          
 132          /* [] END OF FILE */
C51 COMPILER V9.51   S_SCLK_PIN                                                            10/14/2013 23:29:43 PAGE 4   

ASSEMBLY LISTING OF GENERATED OBJECT CODE


             ; FUNCTION _s_sclk_pin_Write (BEGIN)
                                           ; SOURCE LINE # 35
;---- Variable 'value' assigned to Register 'R7' ----
                                           ; SOURCE LINE # 36
                                           ; SOURCE LINE # 37
0000 905100            MOV     DPTR,#05100H
0003 E0                MOVX    A,@DPTR
0004 54DF              ANL     A,#0DFH
0006 FE                MOV     R6,A
;---- Variable 'staticBits' assigned to Register 'R6' ----
                                           ; SOURCE LINE # 38
0007 EF                MOV     A,R7
0008 C4                SWAP    A
0009 33                RLC     A
000A 5420              ANL     A,#020H
000C 4E                ORL     A,R6
000D F0                MOVX    @DPTR,A
                                           ; SOURCE LINE # 39
000E 22                RET     
             ; FUNCTION _s_sclk_pin_Write (END)

             ; FUNCTION _s_sclk_pin_SetDriveMode (BEGIN)
                                           ; SOURCE LINE # 56
;---- Variable 'mode' assigned to Register 'R7' ----
                                           ; SOURCE LINE # 57
                                           ; SOURCE LINE # 58
0000 EF                MOV     A,R7
0001 540E              ANL     A,#0EH
0003 FF                MOV     R7,A
0004 905005            MOV     DPTR,#05005H
0007 E0                MOVX    A,@DPTR
0008 54F1              ANL     A,#0F1H
000A 4F                ORL     A,R7
000B F0                MOVX    @DPTR,A
                                           ; SOURCE LINE # 59
000C 22                RET     
             ; FUNCTION _s_sclk_pin_SetDriveMode (END)

             ; FUNCTION s_sclk_pin_Read (BEGIN)
                                           ; SOURCE LINE # 80
                                           ; SOURCE LINE # 81
                                           ; SOURCE LINE # 82
0000 905101            MOV     DPTR,#05101H
0003 E0                MOVX    A,@DPTR
0004 5420              ANL     A,#020H
0006 7E00              MOV     R6,#00H
0008 7805              MOV     R0,#05H
000A         ?C0005:
000A CE                XCH     A,R6
000B C3                CLR     C
000C 13                RRC     A
000D CE                XCH     A,R6
000E 13                RRC     A
000F D8F9              DJNZ    R0,?C0005
0011 FF                MOV     R7,A
                                           ; SOURCE LINE # 83
0012         ?C0003:
0012 22                RET     
             ; FUNCTION s_sclk_pin_Read (END)
C51 COMPILER V9.51   S_SCLK_PIN                                                            10/14/2013 23:29:43 PAGE 5   


             ; FUNCTION s_sclk_pin_ReadDataReg (BEGIN)
                                           ; SOURCE LINE # 100
                                           ; SOURCE LINE # 101
                                           ; SOURCE LINE # 102
0000 905100            MOV     DPTR,#05100H
0003 E0                MOVX    A,@DPTR
0004 5420              ANL     A,#020H
0006 7E00              MOV     R6,#00H
0008 7805              MOV     R0,#05H
000A         ?C0006:
000A CE                XCH     A,R6
000B C3                CLR     C
000C 13                RRC     A
000D CE                XCH     A,R6
000E 13                RRC     A
000F D8F9              DJNZ    R0,?C0006
0011 FF                MOV     R7,A
                                           ; SOURCE LINE # 103
0012         ?C0004:
0012 22                RET     
             ; FUNCTION s_sclk_pin_ReadDataReg (END)



MODULE INFORMATION:   STATIC OVERLAYABLE
   CODE SIZE        =     66    ----
   CONSTANT SIZE    =   ----    ----
   XDATA SIZE       =   ----    ----
   PDATA SIZE       =   ----    ----
   DATA SIZE        =   ----    ----
   IDATA SIZE       =   ----    ----
   BIT SIZE         =   ----    ----
   EDATA SIZE       =   ----    ----
   HDATA SIZE       =   ----    ----
   XDATA CONST SIZE =   ----    ----
   FAR CONST SIZE   =   ----    ----
END OF MODULE INFORMATION.


C51 COMPILATION COMPLETE.  0 WARNING(S),  0 ERROR(S)
